:10010200120100020000004005168080000001027A
:020112000001EA
:0A0116000A0600020000004001008C
:100122000902270001010080320904000003FF00D8
:10013200000007058102400000070582020002005C
:07014200070588020002001E
:10014A000902270001010080320904000003FF00B0
:10015A0000000705810240000007058202400000F6
:07016A0007058802400000B8
:100172001403000000000000000000000000000066
:10018200000000000C0341004300430045005300FF
:100192001E035700410054004300480044004F0032
:1001A2004700000000000000000000000000000006
:0A3022000001020203030404050587
:1021E700EC4EFEED4F2422F58274303EF583E493E6
:1021F700FF3395E0FEEF24A1FFEE34E68F82F583EF
:102207002290E6BCE0547EFF7E00E0D394807C0001
:1022170022F0E52C2401FFE4352BFEE4352AFDE40A
:1022270035298F2C8E2B8D2AF52922AF30AE2FAD75
:102237002EAC2DAB2CAA2BA92AA829C3020807E587
:0C22470036252CF582E535352BF5832279
:10191F00E4F534F533F532F531C23CC239C23BC27E
:10192F003A1224387E017F028E0A8F0B75120175D1
:10193F00131675080175092275100175114A751472
:10194F0001751572EE54E07003021A0B75350075B0
:10195F0036808E378F38C374B09FFF74019ECF24AB
:10196F0002CF3400FEE48F308E2FF52EF52DF52C9F
:10197F00F52BF52AF529122232500A12224674CD80
:10198F0012221880F1E4F52CF52BF52AF5291222F5
:10199F00325017E538252CF582E537352BF583E0E6
:1019AF00FF122246EF12221880E485350A85360B86
:1019BF0074022480FF740134FFFEC3E5139FF513F7
:1019CF00E5129EF512C3E50D9FF50DE50C9EF50C86
:1019DF00C3E50F9FF50FE50E9EF50EC3E5099FF5C5
:1019EF0009E5089EF508C3E5119FF511E5109EF571
:1019FF0010C3E5159FF515E5149EF514D2E843D8ED
:101A0F002090E668E04409F090E65CE0443DF0D2B7
:101A1F00AFD241122BA190E680E054F7F0538EF82D
:101A2F00C23C303A0512133CC23A303C2912308581
:101A3F005024C23C122C9E20391690E682E030E7EB
:101A4F0004E020E1EF90E682E030E604E020E0E4FD
:0B1A5F00122BD012308712008080C7CD
:10133C0090E6B9E012086513E000143401148E0332
:10134C00135F0613DA0813D40913C80A13CE0B0063
:10135C000014C512307D40030214D190E6BBE0248A
:10136C00FE602214603324FD601114602224067088
:10137C0048E50A90E6B3F0E50B8037E51290E6B34A
:10138C00F0E513802DE50C90E6B3F0E50D8023E538
:10139C000E90E6B3F0E50F801990E6BAE0FF122B41
:1013AC00FCAA06A9077B01EA494B600DEE90E6B357
:1013BC00F0EF90E6B4F00214D10214CA12304002DD
:1013CC0014D11230360214D1122DAE0214D11230B7
:1013DC002C0214D112307F40030214D190E6B8E0F5
:1013EC00247F60151460192402703AA239E4332565
:1013FC00E0FFA23BE4334F8018E490E740F0801606
:10140C0012220840047D0180027D001221E7E05485
:10141C000190E740F0E4A3F090E68AF090E68B743C
:10142C0002F00214D10214CA12308140030214D10A
:10143C0090E6B8E024FE6016240260030214D190FA
:10144C00E6BAE0B40105C2390214D10214CA90E61E
:10145C00BAE0702C12220840047D0180027D00123B
:10146C0021E7E054FEF090E6BCE0548013131354D3
:10147C001FFFE0540F2F90E683F0E04420F08045EE
:10148C00803C123083503E90E6B8E024FE601A2473
:10149C0002703290E6BAE0B40104D239802790E6AB
:1014AC00BAE0B40202801E801512220840047D01AD
:1014BC0080027D001221E78008121E24500790E65E
:0C14CC00A0E04401F090E6A0E04480F0B5
:0114D80022F1
:0300330002307622
:0430760053D8EF320A
:102D2F00E4FFFE7D807C471201B5020401E4FBFA4B
:102D3F00903F801208180202ADE6FE08E6F58BEE12
:032D4F00F58D22DD
:102322008F428E418D408C3FE4FFFEFDFCAB42AA02
:0F23320041A940A83F74E012034C7003C28E22F1
:10234100E589540F4410F589538EEF794078411295
:102351002D3CAB42AA41A940A83F1202AD8F468E47
:10236100458D448C43AB46AA45A944A843122D2F61
:1023710078A1A60608A607C28E18122D48D2ABD2A4
:012381008ECD
:012382002238
:0826A2008F428E418D408C3FF8
:1026AA0079807840122D3CAB42AA41A940A83F123A
:1026BA0002ADAB07AA06A905A804122D2FAD07ACD7
:1026CA0006E4F5C8438E20AF04ECF5CB8FCDAF05F9
:0B26DA00EDF5CA8FCCD2BDD2ADD2CA44
:0126E50022D2
:03001B00022D9023
:102D9000C0E0C0D075D000C000C00678A1122D4898
:0E2DA000A291B39291D006D000D0D0D0E032F4
:03002B000226E6C4
:1026E600C0E0C0F0C083C082C085C084C086758645
:1026F60000C0D075D000C000C003C004C005C0062D
:10270600C007122C28C2CFD007D006D005D004D0DF
:1027160003D000D0D0D086D084D085D082D083D0CC
:04272600F0D0E032DD
:1022BC00456E61626C652041444300446973616200
:1022CC006C652041444300414343455320504349EE
:1022DC00652D5744472D43534D41204331002D5319
:1022EC003031204D6F646500504349652D5744478C
:1022FC002D43534D4100504349652D5744472D43C1
:10230C00534D00414343455320504349652D574499
:06231C00472D3F3F3F008A
:0F2F3A00C13FC13D018CFFC13E011C00011D6460
:1017C300E6FF7843E475F001120855EF0207701243
:1017D30007707843E475F001020855FFAE3F053FFB
:1017E30074402EF582E434E7F58322EE75F003A40A
:1017F3002410F582E4343FF5832290E6BDE0FE90A9
:10180300E6BCE02400FDEC3EFC90E6BFE0FE90E683
:10181300BEE07A002400FBEA3EFA22E090E740F0C3
:10182300E490E68AF090E68B22E5801313543F227E
:10183300EE75F003A42412F582E4343FF5832225E8
:101843003AF53AE53D3539F539C3E53C953EF53C86
:10185300E53B953DF53B227586005391EF90E65DA0
:101863002274402540F58274E7353FF58322AD3E6F
:101873007AE779407F40AB072290E6BBE0FE90E633
:10188300BAE07C002400FFEC3EFE22C3E540953E17
:10189300E53F953D22E490E68AF090E6BEE090E6CF
:1018A3008BF02275F003A42411F582E4343FF58311
:1018B3002290E68AE53EF090E68BE53DF022E53A9C
:1018C3002540F582E539353FF5832274002539F942
:1018D300EE34FCFA7B0122F582E4343FF583228562
:1018E3000D82850C83A37402F022850F82850E83FB
:1018F300A37407F0227D017B007E00020974D3E507
:101903003E9400E53D940022D3E53E9400E53D94EA
:0C1913000022087601087601E408F622A4
:0F2F6E0090E6C2E02041044402F02254FDF0221C
:0F2F7D0090E6C2E02041044401F02254FEF0220D
:0F2F8C0090E6C2E02041044404F02254FBF022FE
:0F2F9B0090E6C2E02040044402F02254FDF022F0
:0F2FAA0090E6C2E02040044401F02254FEF022E1
:0F2FB90090E6C2E02040044404F02254FBF022D2
:07306300EFF490E6C2F02239
:03307A00D29522CA
:102F0200D295E4FFFE0FBF00010EBE04F8BFB0F57C
:022F1200C29566
:012F1400229A
:06276D008B408A41894205
:102773008B438A44894578431217D7E523120770A0
:1027830090E685E0FF78431217D7EF12077090E6C3
:1027930084E0FF78431217D7EF12077078431217BC
:0B27A300D7ED120770C3E5459542FF1B
:0127AE002208
:062160008B408A41894218
:102166008B438A4489451217D5E5231217D2E522F7
:102176001217D2E5211217D2E525120770789C12A4
:1021860017C3789B1217C3787A1217C37879121778
:10219600C378701217C3786F1217C378721217C3F9
:1021A60078711217C378741217C378731217C3782D
:1021B600761217C378751217C31217D5E5241207BE
:1021C60070787B1217C3788B1217C3788D1217C3DA
:1021D60078771217C378781217C3C3E5459542FF7F
:0121E60022D6
:0527AF00E5AA30E63A46
:1027B4007539017E001218CE789AE6FD12276DEF66
:1027C4002539F539E4789AF61218CE122160EF25EE
:1027D40039F539E4787BF6F52490FC00E539F0907E
:0A27E400E69C7402F0E490E69DF01C
:0127EE0022C8
:07306A00EF4480789AF62282
:072B7200AD07E5AA30E027E2
:102B7900753F017E007400253FF9EE34F0FA7B01C0
:102B890012276DEF253FF53F90F000F090E6907425
:072B990002F0E490E691F068
:012BA0002212
:102EEE00200710D207D23EC2007F01122B727F053F
:042EFE00121D64221B
:0F2FC800203D0BD23DD294D2077F06121D64220A
:10299600EF30E505903F02EDF0EF30E405903F03A0
:1029A600EDF0EF30E305903F09EDF0EF30E20590F2
:1029B6003F08EDF0EF30E105903F07EDF0EF30E036
:0729C60005903F06EDF02231
:101EB2008F3F7440C3953F50047F408002AF3FEF95
:101EC200C39418500F7440C3953F50047F4080065E
:101ED200AF3F80027F188F3F78407CE77A00797CA1
:101EE2007F0E1218F8784D7CE77A0079907F0A12FB
:0E1EF20018F890E7407418121822E53FF0220D
:101663008E398F3A8C3B8D3C8A3D8B3E90E6B8E0B9
:1016730030E7030217B8122F28121901403312184A
:101683009890E6A0E020E1F9E53E640E453D600355
:101693000217C2C2AFAE3DAF3E787C7C00FD7B013A
:1016A3007AE77940120974D2AF787EE6FF7E008034
:1016B30053E53C853BF012088B17110001173300EB
:1016C300021703004416F3004916F8004A16F00007
:1016D30052170A005416FD00691700006A17368076
:1016E300001754800117A48002000017C2022F5D67
:1016F300E4FF022B727F0202306A022E9A022EAF9F
:10170300AF3AAE39022C50AF3AAE390230003087CF
:10171300030217C2E539453A24FFB39282E53A45FD
:101723003970047F0180027F00EF24FFB3923F22D0
:101733000224DDE4FBFD7F08122E577F007E007D2F
:10174300007C00122322308705C290C29122C291ED
:1017530022308733E539700EC291FBFD7F08122ECC
:1017630057C291C29022E539FFBF0105308613802D
:101773000CEF64027049E53AC394805005C290D2DD
:101783009122C291D29022E539FFBFFF09E53AFBCE
:101793007DFF7F08801CAC39AD3AE41203C80223F5
:1017A30022C3E539948040047F0980027F0A7B507D
:1017B3007D02022E571219014005AF3E121EB222BE
:101C73008F398D3A8B3B90E6B8E030E703021D07BE
:101C8300E53D7074E53E7070E53C7F00FEEF253B5B
:101C9300FFE43EFEEF8EF012088B1CD900001CDE21
:101CA30000011CE801001CE801011CE801021CE81A
:101CB30001031CE801041CE801051CE801061CE8FB
:101CC30001071CE801081CE801091CE8010A1CF1D2
:101CD300FFFF00001D63AF390229CDE539FD7C000C
:101CE300AF3A021FB8AB39AD3AAF3B022E57E53AD4
:101CF300606EAD39FF0229961218B490E6A0E03069
:0B1D0300E15E80F7E53DD39400405501
:101D0E00753F017440253FF9E434E7FA7B017DFF0E
:101D1E0012276DEF253FF53F2440F9E434E7FA7BB7
:101D2E0001122160EF253FF53FE4787BF6F524E5BF
:101D3E003BB4010C12282FAE3F053F1217E3EFF014
:101D4E0090E740E53FF01218B4E53A7008E539B473
:051D5E000103122FE556
:011D6300225D
:101E240090E6B9E01208651E4D101E4D111E6A4061
:101E34001EA9A21EA9A31E7DD41E90D51E97D61E30
:101E44009CD71EA4D800001EAE90E6BAE0FFA3E023
:101E5400FDA3E0FBA3E0F53CA3E0F53DA3E0F53EE4
:101E6400121C73021EB012187CC006C0071217FDA4
:101E7400D007D006121663803312187CC006C00740
:101E84001217FDD007D006120EDE80207F01122B20
:101E94007280081227AF800312257D122F28800C30
:0E1EA400122C9E8007121B728002D322C322D2
:100EDE008E398F3A8C3B8D3C8A3D8B3E90E6B8E046
:100EEE0030E7030210A112190B400A12189890E66F
:100EFE00A0E020E1F9E53A8539F012088B0F8B005E
:100F0E0001100100A00FCC00B00F9700D0103001DF
:100F1E00A0102A01A1102401A2101E01A310180175
:100F2E00A4101201A5100C01A6100601A70FFB01BB
:100F3E00B00FF501B10FEF01B20FE901B30FE301ED
:100F4E00B40FDD01B50FD701B60FD101B70FC60132
:100F5E00D00FC001D10FBA01D20FB401D30FAE0121
:100F6E00D40FA801D50FA201D60F9C01D71036FFC2
:100F7E00001071FF011093FF020000133BE53C547B
:100F8E000175F011A490E6C2F0E53CF5B022E53C07
:100F9E001392B722E53C1392B622E53C1392B5228A
:100FAE00E53C1392B422E53C1392B322E53C139236
:100FBE00B222E53C1392B122E53C1392B022E53CFD
:100FCE00F59022E53C13929722E53C13929622E58A
:100FDE003C13929522E53C13929422E53C13929396
:100FEE0022E53C13929222E53C13929122E53C13AA
:100FFE00929022E53CF58022E53C13928722E53C57
:10100E0013928622E53C13928522E53C13928422AC
:10101E00E53C13928322E53C13928222E53C139227
:10102E008122E53C1392802212190B500302133BCE
:10103E00AE3DAF3E7C007D031207A4ED4C60030273
:10104E00133BD3E53E9430E53D9400400302133B41
:10105E00AE3DAF3E78107C3F7D017B017AE7794053
:10106E00020974AF3CE53CBF010D122F02D23F7B4B
:10107E00FF7A2279BC800B12307AC23F7BFF7A2234
:10108E0079C70227EFAF3CBF0103D38001C3924162
:10109E00023071E53A8539F012088B1315000213F0
:1010AE002E0003123900A011B100B0112900D01288
:1010BE00B101A012A101A1129101A2128101A312EC
:1010CE007101A4126101A5125101A6124101A712CC
:1010DE002901B0121901B1120901B211F901B311AE
:1010EE00E901B411D901B511C901B611B901B71190
:1010FE00A101D0119101D1118101D2117101D31130
:10110E006101D4115101D5114101D6113101D7120E
:10111E00C1FF0012D6FF010000133B90E740E5B07F
:10112E0002133430B7047F0180027F0090E740EF56
:10113E0002133430B6047F0180027F0090E740EF47
:10114E0002133430B5047F0180027F0090E740EF38
:10115E0002133430B4047F0180027F0090E740EF29
:10116E0002133430B3047F0180027F0090E740EF1A
:10117E0002133430B2047F0180027F0090E740EF0B
:10118E0002133430B1047F0180027F0090E740EFFC
:10119E0002133430B0047F0180027F0090E740EFED
:1011AE0002133490E740E5900213343097047F0128
:1011BE0080027F0090E740EF0213343096047F01E7
:1011CE0080027F0090E740EF0213343095047F01D8
:1011DE0080027F0090E740EF0213343094047F01C9
:1011EE0080027F0090E740EF0213343093047F01BA
:1011FE0080027F0090E740EF0213343092047F01AB
:10120E0080027F0090E740EF0213343091047F019B
:10121E0080027F0090E740EF0213343090047F018C
:10122E0080027F0090E740EF02133490E740E580A4
:10123E000213343087047F0180027F0090E740EF75
:10124E000213343086047F0180027F0090E740EF66
:10125E000213343085047F0180027F0090E740EF57
:10126E000213343084047F0180027F0090E740EF48
:10127E000213343083047F0180027F0090E740EF39
:10128E000213343082047F0180027F0090E740EF2A
:10129E000213343081047F0180027F0090E740EF1B
:1012AE000213343080047F0180027F0090E740EF0C
:1012BE00021334AE3DAF3E78407CE77D017B017A70
:0812CE003F79101209748051F0
:1012D600E4F53F789FE6FE08E6FDAC3F053F744027
:1012E6002C1217E6EDF0EE1217DEEFF01217DFE51F
:1012F6001FF0E51E1217DEEFF0C3E53F953EE495BD
:0F1306003D5004AF3F8002AF3E90E68BEFF022E8
:1013150090E6F4E020E1047F0180027F0090E74041
:10132500EFF090E68BE53EF02212182C90E740F0A6
:0713350090E68B7401F02229
:102F2800C2AFE4F51EF51FD2AFC23DD2007F040246
:022F38001D6416
:0D2FF300C2AF051FE51F7002051ED2AF2200
:0C300000C2AFEF787FF6EE08F6D2AF22E8
:1014D900AF23E5805403C454F0FEE5B0540F4EF534
:1014E90023E5236F787B46F6A21B301301B3502501
:1014F900903F0FE014F0E07024A21B301301B37287
:10150900239223A21B9213A213720B920BA22BA05C
:1015190013922B8000903F09E0903F0FF0A21A3000
:101529001201B35025903F0EE014F0E07024A21A86
:10153900301201B372229222A21A9212A212720AD4
:10154900920AA22AA012922A8000903F08E0903FB6
:101559000EF0A219301101B35025903F0DE014F09F
:10156900E07024A219301101B372219221A21992BB
:1015790011A21172099209A229A011922980009041
:101589003F07E0903F0DF0A218301001B3502590AD
:101599003F0CE014F0E07024A218301001B372205F
:1015A9009220A2189210A21072089208A228A010E4
:1015B90092288000903F06E0903F0CF0A21D301564
:1015C90001B35025903F05E014F0E07024A21D30CE
:1015D9001501B372259225A21D9215A215720D92BD
:1015E9000DA22DA015922D8000903F03E0903F059C
:1015F900F0A21C301401B35025903F04E014F0E030
:101609007024A21C301401B372249224A21C9214D7
:10161900A214720C920CA22CA014922C8000903F60
:1016290002E0903F04F0788BE655245522788D46E8
:10163900F67877E65524FFE522F45F0846F6788ABE
:10164900E6F4552460057F0212306A787BE660056E
:091659007F0212306A788AA6248F
:011662002265
:101FB800EF1208651FE1001FE9011FF1021FF90375
:101FC800200104203705202C06202107200908209D
:101FD800110920190A00002042EC4D24FF92B78015
:101FE8005BEC4D24FF92B58053EC4D24FF92B680F4
:101FF8004BEC4D24FF92978043EC4D24FF92968042
:102008003BEC4D24FF92918033EC4D24FF9293805A
:102018002BEC4D24FF92928023EC4D24FF92411229
:102028002F6E8018EC4D24FF9241122F7D800DEC0D
:0E2038004D24FF9241122F8C8002C322D3222E
:10204600EF120865206F00207701207F02208703AA
:10205600208F0420C50520BA0620AF072097082048
:102066009F0920A70A000020D0EC4D24FF92B780DC
:102076005BEC4D24FF92B58053EC4D24FF92B68065
:102086004BEC4D24FF92978043EC4D24FF929680B3
:102096003BEC4D24FF92918033EC4D24FF929380CC
:1020A6002BEC4D24FF92928023EC4D24FF9240129C
:1020B6002F9B8018EC4D24FF9240122FAA800DEC26
:0E20C6004D24FF9240122FB98002C322D32274
:1029CD00903F10E07005EFA2E392B7903F13E070D7
:1029DD0005EFA2E192B5903F16E07005EFA2E292ED
:1029ED00B6903F19E07004EF139297903F1CE07082
:0729FD0005EFA2E49296220F
:10282F00E4FF3097047E0180027E00EE420730B550
:10283F00047E0280027E00EE420730B6047E0480E2
:10284F00027E00EE420730B7047E0880027E00EE63
:0E285F0042073096047E1080027E00EE420793
:01286D002248
:10238300EF14601914601F14602914603314603D46
:10239300240570497FE3123053789B803B7FE5121D
:1023A300305378798032C293C2927FEE12305378E1
:1023B3006F8025C293D2927FEE12305378718018CA
:1023C300D293C2927FEE1230537873800BD293D2A2
:0E23D300927FEE1230537875A60608A60722F8
:102F4C00AF1C051C122383E51C75F0068485F01C50
:012F5C002252
:102E8500E4F53FE4FBFDAF3F122E57053FE53FC399
:042E9500941040EF66
:012E99002216
:102E5700AE07C2AF121833EFF01218A6EBF0EF125D
:062E670017EFEDF0D2AF01
:012E6D002242
:10261300E4FE788C061217EEE0D394004034788CF5
:10262300E6FB700E121833E0FF7D017C001220469A
:102633008020EE1218A6E06B7018121833E0FFE446
:10264300FDFC1220461217EEE0F460061217EEE0CE
:0826530014F00EEE641070BDDE
:01265B00225C
:0E2FD700E4F5B275B3FF75B5F090E6C3F022D5
:102924007890760A12191530B1047F0180027F0075
:10293400EF25E025E04463FF30B0047E0180027E91
:1029440000EE25E04FF5207894F6E408F608F678D2
:0929540099F6C294C207C2912257
:10257D0090E61274E0F000000090E615F000000007
:10258D0090E611F000000090E610E0547FF000009E
:10259D000090E613E0547FF000000090E614E05444
:1025AD007FF0000000122E9A122EAF90E683741267
:0C25BD00F07432F090E65CE04402F02282
:0E2FE500E4F521F525F524788DF67878F622AE
:102B0D00903F027401F0903F04F0903F03F0903F2E
:102B1D0005F0903F09F0903F0FF0903F08F0903F87
:102B2D000EF0903F07F0903F0DF0903F06F0903F74
:032B3D000CF02277
:10286E007F07123063E4789DF608F6D200C23EC2AE
:10287E003DC207C297787C760E08760108F608F6F8
:10288E0008F608760108F608F63087047FFF800206
:0E289E007F007884A60712191508F608F622A6
:102438007F01121D6412307A12305B903F01745193
:10244800F0903F0B7401F090E600E054E74410F080
:10245800903F801208244C371B00122A0412295D71
:1024680012257D1224DD43AF017BFF7A2279D31236
:1024780027EF3087097BFF7A2279EA1227EF7F025C
:03248800021D64CE
:10008000D3798FE778A09619E718965005C24112E8
:100090002F6E787EE66034203E177880E6FE18E604
:1000A000FDEDFFD3E51F9FE51E9E401F122EEE8043
:1000B0001A7880E6FE18E6FDEEFCE51EC313FEE5A9
:1000C0001F13D39DEE9C4003122FC8A2809202A260
:1000D000B092037894A620E51F7897F6E51E08F6FF
:1000E000789AE6C3948040031227AF30870A90E6DF
:0F00F000F4E020E003122FC8303F03122F4C2200
:102E9A0090E6047480F00000007402F0000000E480
:052EAA00F00000002211
:102EAF0090E6047480F00000007408F0000000E465
:052EBF00F000000022FC
:102F5D007F007E007D007C0012232212286E022944
:012F6D00243F
:1024DD00E4789AF67F07123063122EAF122E9A7897
:1024ED008B763F7877763FE4788AF6C23DC2B7C2E5
:1024FD0094C207C291122FE5122B0D122E857F006B
:10250D007E007D7A7C441226A2122FD7122F5D30C9
:10251D0087097B507D027F0A122E577F010230639F
:102A0400E4F5391218737D087FF87E1D12252DE434
:102A1400F539744025391217E6E0FDE53975F00201
:102A2400A42474F9740135F08982F583EDF0053935
:052A3400E539B408DDE6
:012A3900227A
:0623E1008B398A3A893BAA
:1023E700E4F53C122ED98F3DE53D25E0240290010E
:1023F70092F0E4F53CAF3DEF3395E0FEC3E53C9F3B
:10240700EE6480F87480985027AB39AA3AA93B85C7
:102417003C82758300120743FDE53C75F002A42456
:1024270094F9740135F08982F583EDF0053C80C598
:012437002282
:10295D001218737D017F037E0012252D90E740E054
:10296D0090010CF090E740E0247F600B0470107B29
:10297D00FF7A2279F4800E7BFF7A23790280067B21
:09298D00FF7A23790F1223E122E5
:09304A00787E76017F03021D640B
:102C5000EF4E60047F0180027F00787EEFF6600413
:102C60007F0380027F07121D64787EE670081218C9
:072C70002C700312300C224E
:102C28001226131214D9D51D1E78A006E6187001B5
:102C380006C378A0E6940A18E694004007122FF31A
:072C4800E4F608F6751D64B7
:012C4F002262
:102EC4007B807DFF7F03122E57D297C241122F7D44
:052ED400C241022F8C39
:0B300C00C2977B80E4FD7F03022E577B
:101D6400EF1208651D81011D9E021DAC031DB904FF
:101D74001DE1051DF2061E140700001E237FFF123D
:101D840029CDE490E6C2F012182C7005D241022F3E
:101D94007D208503021E23021E1C12182C700302D0
:101DA4001E2330857A021E1C12182C7003022EC4C6
:101DB40030856C803512182C70028003308560D217
:101DC40041122F6E78A0E62402FF18E436FE7C0050
:101DD4007D0A1207A4788EA60408A6052212182CE0
:101DE40070057F050230633085357F018017788464
:101DF400E6600B7F007E007DFA7C441223221218D9
:101E04002C70087F04123063D2B722308511800809
:101E140012182C600A3085077F04123063C2B7227F
:102CC300C0E0C083C082C085C084C086758600D240
:102CD3003A12185D7401F0D086D084D085D082D0AA
:042CE30083D0E03288
:102D5200C0E0C083C082C085C084C08612185A7485
:0F2D620004F0D086D084D085D082D083D0E032E8
:102D7100C0E0C083C082C085C084C08612185A7466
:0F2D810002F0D086D084D085D082D083D0E032CB
:102AA500C0E0C083C082C085C084C08675860085AD
:102AB500100C85110D1218E285080E85090F1218E4
:102AC500ED12185D7410F0D086D084D085D082D0F8
:042AD50083D0E03298
:102CE700C0E0C083C082C085C084C086758600D21C
:102CF7003C12185D7408F0D086D084D085D082D07D
:042D070083D0E03263
:1028E900C0E0C083C082C085C084C0867586009060
:1028F900E680E030E71285080C85090D1218E2859B
:10290900100E85110F1218ED12185D7420F0D08683
:0B291900D084D085D082D083D0E03283
:0100FF0032CE
:013089003214
:01308A003213
:01308B003212
:01308C003211
:01308D003210
:01308E00320F
:01308F00320E
:01309000320D
:01309100320C
:01309200320B
:01309300320A
:013094003209
:013095003208
:013096003207
:013097003206
:013098003205
:013099003204
:01309A003203
:01309B003202
:01309C003201
:01309D003200
:01309E0032FF
:01309F0032FE
:0130A00032FD
:0130A10032FC
:0130A20032FB
:0130A30032FA
:0130A40032F9
:0130A50032F8
:0130A60032F7
:0130A70032F6
:0130A80032F5
:0130A90032F4
:0130AA0032F3
:0130AB0032F2
:06272A00AB07AA06AC0596
:10273000E4FD903F0BE0600B7E000DEE2487121845
:10274000DAEAF0AE050D74872E1218DAEBF0AF0559
:102750000D74872F1218DAECF0903F01E0FF7A3FFA
:0D2760007B87122E06903F01E0FF022A3A0F
:0A2A70008E418F428D438A448B454E
:102A7A00E4F546E546C3954350200542E542AE419A
:102A8A007002054114FFE5452546F582E43544F513
:0A2A9A0083E0FD12272A054680D9CB
:012AA400220F
:0A252D008E418F428D438A448B4596
:10253700E4FDF546903F0BE06012E541FF7E000D9C
:10254700EE2487F582E4343FF583EFF0AE050D7492
:10255700872EF582E4343FF583E542F0903F01E0B2
:10256700FF7A3F7B87122E06903F01E0FFAB45AA1B
:0625770044AD43022DEA11
:02307D00D3225C
:102DAE0000000090E6247402F0000000E490E62596
:0E2DBE00F000000090E6BAE0903F0AF0D32249
:0A302C00903F0A12181E04F0D32290
:0A30360090E6BAE0903F00F0D322CC
:0A304000903F0012181E04F0D32286
:02307F00D3225A
:02308100D32258
:02308300D32256
:02308500D32254
:02308700D32252
:101B720090E6BAE0753900F53AA3E0FEEE423990FC
:101B8200E6BEE0753B00F53CA3E0FEEE423B90E68C
:101B9200B8E064C06003021C19E53C453B700302D7
:101BA2001C7290E6A0E020E1F9C3E53C9440E53BDD
:101BB20094005008853B3D853C3E8006753D00758E
:101BC2003E4090E6B9E0B4A31EE4F53FF54012189A
:101BD2008E50381218C1E0FF121864EFF00540E58C
:101BE2004070EB053F80E7E4F53FF54012188E5058
:101BF2001012186474CDF00540E54070EF053F8087
:101C0200EB121871AF3AAE3912252D121823E53EA8
:101C1200F0121842021B9B90E6B8E064407051E556
:101C22003C453B604B121823F090E6A0E020E1F91E
:101C320090E68BE0753D00F53E90E6B9E0B4A31E58
:101C4200E4F53FF54012188E501E121864E0FF12A0
:101C520018C1EFF00540E54070EB053F80E7121830
:101C620071AF3AAE39122A70E53E121842021C21B7
:011C7200224F
:03004300021F0099
:03005300021F0089
:101F0000022CC300022D7100022D5200022CE700AA
:101F1000022AA5000228E9000200FF000230890021
:101F200002308A0002308B0002308C0002308D00BB
:101F300002308E0002308F0002309000023091009B
:101F40000230920002308900023093000230940087
:101F5000023095000230960002309700023098005F
:101F60000230990002308900023089000230890075
:101F700002309A0002309B0002309C0002309D002B
:101F800002309E0002309F000230A0000230A1000B
:101F90000230A2000230A3000230A4000230A500EB
:101FA0000230A6000230A7000230A8000230A900CB
:081FB0000230AA000230AB0070
:022D0B008F6EC9
:102D0D00903F86EDF07A3F7B867D01122E067A3F4D
:102D1D007B847D02AF6E122DEA903F84E0FEA3E02E
:012D2D00FFA6
:012D2E002282
:1028AC00AE07C2E990E678E04480F0EE25E090E6D1
:1028BC0079F090E678E030E0F9ED90E679F090E68A
:1028CC0078E030E0F990E678E04440F090E678E08B
:0D28DC0030E0F990E678E020E6F9D2E9223C
:022E6E00AC07AF
:102E70001228AC7A3F7B877D02122DEA903F87E0D3
:042E8000FEA3E0FFCE
:012E8400222B
:08305300AD077F40122E6E2232
:102BD00090E682E030E004E020E60B90E682E03010
:102BE000E119E030E71590E680E04401F07F147EC3
:0C2BF0000012265C90E680E054FEF0220B
:102C9E0090E682E044C0F090E681F04387010000A8
:042CAE000000002200
:102BA10030410990E680E0440AF0800790E680E039
:102BB1004408F07FDC7E0512265C90E65D74FFF030
:0F2BC10090E65FF05391EF90E680E054F7F0223A
:08305B00E4F51BD2E9D2AF221B
:102A3A0090E678E020E6F9C2E990E678E04480F092
:102A4A00EF25E090E679F090E678E030E0F990E65C
:102A5A0078E04440F090E678E020E6F990E678E005
:062A6A0030E1D6D2E922A2
:102B4000A90790E678E020E6F9E51B702390E67887
:102B5000E04480F0E925E090E679F08D16AF03A916
:102B6000077517018A188919E4F51A751B01D32214
:022B7000C3227E
:102AD900A90790E678E020E6F9E51B702590E678ED
:102AE900E04480F0E925E0440190E679F08D16AFE5
:102AF90003A9077517018A188919E4F51A751B03C3
:042B0900D322C322EE
:03004B00021A6A2C
:101A6A00C0E0C083C082C085C084C086758600C0BD
:101A7A00D075D000C000C001C002C003C006C007B4
:101A8A0090E678E030E206751B06021B5490E67871
:101A9A00E020E10CE51B64026006751B07021B547B
:101AAA00E51B24FE605F14603624FE7003021B45AA
:101ABA0024FC7003021B5124086003021B54AB1759
:101ACA00AA18A919AF1A051A8F827583001207433B
:101ADA0090E679F0E51A65167070751B05806B90B3
:101AEA00E679E0AB17AA18A919AE1A8E8275830097
:101AFA00120782751B02E5166401704E90E678E0C3
:101B0A004420F08045E51624FEB51A0790E678E0F1
:101B1A004420F0E51614B51A0A90E678E04440F03D
:101B2A00751B0090E679E0AB17AA18A919AE1A8EB0
:101B3A0082758300120782051A800F90E678E044C6
:101B4A0040F0751B008003751B005391DFD007D04E
:101B5A0006D003D002D001D000D0D0D086D084D015
:081B6A0085D082D083D0E03267
:022BFC00A90727
:102BFE00AE14AF158F828E83A3E064037017AD0100
:102C0E0019ED7001228F828E83E07C002FFDEC3E49
:092C1E00FEAF0580DF7E007F009F
:012C2700228A
:102DEA00122AD9E51B24FA600E146006240770F330
:0C2DFA00D322E4F51BD322E4F51BD32206
:102E0600122B40E51B24FA600E146006240770F3AB
:0C2E1600D322E4F51BD322E4F51BD322E9
:10265C008E398F3A90E600E054187012E53A240156
:10266C00FFE43539C313F539EF13F53A801590E6CD
:10267C0000E05418FFBF100BE53A25E0F53AE539B8
:10268C0033F539E53A153AAE39700215394E600515
:06269C00122CB280EE22B8
:102CB2007400F58690FDA57C05A3E582458370F935
:012CC20022EF
:0B30170025303262580025303458008C
:022F4900C14283
:102E3E00743FF59A7440F59B74E7F59D74C0F59E4A
:092E4E00E4227B017A3F79402265
:05307100A24192422281
:1025C900204204E4FEFF2290E6A2E020E1F9122E67
:1025D90050122ED9EF2401F544E43EF543122E3E64
:1025E900FFFEC3EF9544E5436480F8EE648098509C
:1025F9000F90E67BE090E67CF00FBF00010E80E2D1
:09260900E54490E68FF0AE43FFBA
:0126120022A5
:1027EF008B408A418942204204E4FEFF22122825B1
:1027FF008E498F4A854046854147854248122E5063
:10280F0012248B12282574402FF582743F3EF583D6
:10281F00E4F01225C922AB40AA41A942122ED922B7
:102F1500204204E4FEFF22903F40EFF0E4A3F012CC
:032F250025C92299
:102E2200204204E4FEFF227550FF7551307552179F
:0C2E32008F53122E50120ACB1225C92219
:102DCC00204204E4FEFF227550FF75513075521DF0
:0E2DDC008E538F54122E50120ACB1225C9228C
:1022530090E685E02405F569204204E4FEFF227838
:10226300407C3F7D01120A5290E6A2E030E10790E4
:06227300E685E0B569F20A
:10227900122E50122ED9EF2401F56DE43EF56C12A1
:102289002E3EF56AF56BC3E56B956DE56C6480F8D8
:10229900E56A648098501290E67BE090E67CF00550
:1022A9006BE56B70E1056A80DDE56D90E68FF0AE58
:0222B9006CFFB8
:0122BB002200
:1001B20002046DE86480F8E933E83360110460F00A
:1001C200ED33EC337009E8FCE9FDEAFEEBFF2204B3
:1001D20060DED3EB9FEA9EE99DE8C2E78CF0C2F7AE
:1001E20095F0400CE8CCF8E9CDF9EACEFAEBCFFB7A
:1001F20012043885D0F05804700320D5B3E8047097
:10020200075002B2D502047792D5EC0460F7E4CC31
:10021200C0E0C398F8603B94186008400DD0E0FB42
:1002220002044FE4FBFAC9FC8028E830E406E4C982
:10023200FBE4CAFCE830E305E4C9CACBFCE8540796
:100242006010F8C3E913F9EA13FAEB13FBEC13FCA1
:10025200D8F130F52FC3E49CFCEF9BFFEE9AFEED44
:1002620099FDD0E0FBEF4E4D4C701222DB030204ED
:1002720074EC2CFCEF33FFEE33FEED33FDED30E793
:10028200EB02044FEF2BFFEE3AFEED39FDD0E0FB1F
:1002920050130BBB0003020477ED13FDEE13FEEFC8
:0802A20013FFEC13FC02044FF2
:1002AA00020477EC5D046005E85904700302046DEA
:1002BA00120438580460F6EC4860F2EC7004FDFE53
:1002CA00FF22C860DB2481C85009C3986002500627
:1002DA000204749850CAF582E9294B4A7005AB8228
:1002EA0002046375F0007C1A7880C3EF9BEE9AEDE6
:1002FA0099400DC3EF9BFFEE9AFEED99FDE842F09F
:10030A00DC23ACF0D0E0FFD0E0FED0E0FDAB8220F1
:10031A00E7101BEB60BAEC2CFCEF33FFEE33FEED7B
:10032A0033FD02044FE803F830E705C0F075F0002A
:10033A00EF2FFFEE33FEED33FD40B830E7C280AA5F
:10034A0074F8CC6480CCC86480C8F58204604FC35A
:10035A00EB9FF5F0EA9E42F0E99D42F0E89C45F0F9
:10036A00603C501DE5825FFFE582D313CB5BCBF483
:10037A002B5582FB50280ABA002409B900200880AC
:10038A001DE5825BFBE582D313CF5FCFF4C3132F46
:10039A005582FF50090EBE00050DBD00010CC3EBCE
:1003AA009FF5F0EA9E42F0E99D42F0E89C45F06034
:0903BA0007CC4820E701B3EC2256
:1003C30075F020800E75F010800575F0087D007EB5
:1003D300007F003392D530D5031207F9EC33401078
:1003E300EF33FFEE33FEED33FDEC33FCD5F0ED22BE
:0E03F300E5F0247EA2D513CC92E7CDCEFF22FA
:10040100EDD2E7CD33EC3392D524814006E4FFFEF3
:10041100FDFC22FCE4CFCECDCC24E0501174FF8052
:10042100EDC3CC13CCCD13CDCE13CECF13CF0470EF
:07043100F030D5DE0207F9EF
:100A6F00E5642450F8E6056422784D30370278505B
:100A7F00E475F00112085502072A2030EB7F2ED2C1
:100A8F00308018EF540F2490D43440D4FF30340BFF
:100A9F00EF24BFB41A0050032461FFE5656002150F
:100AAF00650568E5687002056730370D784DE475A8
:100ABF00F001120855EF020770022C777403D2373A
:100ACF008003E4C237F5648B4D8A4E894FE4F56598
:100ADF00F567F568E56560077F20120AAA80F5754E
:100AEF0066FFC231C230C232C233C235C236C238DB
:100AFF00120A78FF700D3037057F00120ABBAF68FE
:100B0F00AE6722B4255FC2D5C234120A78FF24D053
:100B1F00B40A00501A75F00A786530D50508B6FF8B
:100B2F000106C6A426F620D5047002D23380D9243C
:100B3F00CFB41A00EF5004C2E5D234020DA8D2315F
:100B4F0080C6D23080C0D23280BCD2D580BAD235E6
:100B5F0080B47F20120AAA2032077401B5650040C5
:100B6F00F1120A6FFF120AAA020AE3D238D23680B4
:100B7F0095120A6FFB120A6FFA120A6FF94A4B703D
:100B8F0006799F7A0E7BFF20322EE565602A7E0064
:100B9F008E8275830012074360060EEE656670F055
:100BAF00C2D5EBC0E0EAC0E0E9C0E0EE120E08D01B
:100BBF00E0F9D0E0FAD0E0FB12072AFF60AAEBC001
:100BCF00E0EAC0E0E9C0E0120AAAD0E02401F9D0BF
:100BDF00E03400FAD0E0FBE5660460DCD566D9802E
:100BEF0087D23280A2120DEB60F7E5667001041216
:100BFF000482A966600DE566600914F566120E920F
:100C0F00EF60F3EA30E702F404C3995077EAF42572
:100C1F00660430E701E404F566800D120DEB60C148
:100C2F00EA05662566120482EA7863F630E701E486
:100C3F00256604D5660420350114120E08E4C0E0C1
:100C4F00120E927863E6601320E70714F6120A92E9
:100C5F00802204F6D0E014C0E07F00120A92E5660D
:100C6F006007120A891566800B303503120A89D086
:100C7F00E0020AE3D0E00480C5120DEB60A0E56648
:100C8F00041204827863EAF6E566203502600104F7
:050C9F002404120E0800
:100CA40074FF04C0E0120E92120A92E56620350227
:100CB4006003120A89D0E0B566E87F45120A9C7881
:100CC40063E67F2B30E7047F2DF404C0E0120AAA08
:100CD400D0E075F00A84C0F0120A93D0E0120A93AF
:100CE400020AE3791080027908C236C2388008D239
:100CF400D5790A8004790AC2D5E566047002F566DE
:100D0400E4FAFDFEFF120A6FFC7B08203113120A7D
:100D14006FFD7B1030300A120A6FFE120A6FFF7BE0
:100D240020EC3382D592D55013C3E43030069FFFB4
:100D3400E49EFEE42031039DFDE49CFCE4CBF8C278
:100D440031EC700CCFCECDCCE824F8F870F38017DA
:100D5400C3EF33FFEE33FEED33FDEC33FCEB33FB3B
:100D6400994002FB0FD8E9EB303105F8D0E0C448D4
:100D7400B231C0E00AEC4D4E4F78207B0070C2EADD
:100D8400B5660040BCC0E0120E0AD0F0D0E02031BD
:100D940004C4C0E0C4B231C0F0120A93D0F0D5F05C
:100DA400EB020AE31208650B80530CE7580B514C15
:100DB4000B4D420CEB4F0CF3440CF3490B66430C04
:100DC400F9550C2A460C88450BF4470EBF500B55B9
:100DD4002D0B592E0B7C2B0B5D230B7A200EA82A8E
:100DE4000B154800000B74E566B4FF037566061224
:100DF4000A6FFC120A6FFD120A6FFE120A6FFF7867
:100E04005C0204B1790AA2D5203314303509B91033
:100E1400020404B9080104A2D520360250010420BA
:100E240032689232B565005034C0E07F2030331907
:100E34007F30A23272367235500F120E61C232C246
:100E440036C235C2387F30800F303503E9C0E01236
:100E54000AAA303503D0E0F9D0E0B565CC303517B7
:100E64007F30B9100C120AAA7F583034077F78807B
:100E740003B90803120AAA3032057F2D020AAA7F99
:100E8400202038F87F2B2036F322923280CF7F0047
:100E9400B407005005245CF8E6FF22286E756C6CDC
:100EA4002900D231120A6F3031F8C231786530D559
:100EB4000108F6020B152D50434958120A6F2403FA
:100EC400B405004001E4900EBA93120A9B743A12DE
:0A0ED4000A9BD233756504020CE797
:10043800E9D2E7C933E833F892D5EDD2E7CD33EC0A
:0704480033FC5002B2D52283
:10044F00EC30E7100FBF000C0EBE00080DBD00040E
:10045F000BEB6014A2D5EB13FCED92E7FD2274FFBA
:10046F00FCFDFEFF22E480F8A2D574FF13FC7D8013
:03047F00E480EF27
:10048200F920E72824F950037907E4F42402FB1841
:10049200DBFDE624FB5014E9600DE4F618E604F6F1
:0F04A200B40A08E4F6D9F57401F60A22C2D5228D
:1004B100ED33EC3392D5FA602AB4FF33EDC2E77B1A
:1004C100FF60067A0479D6E4227A0479DF20D50424
:1004D1007A0479DA224E614E002B494E46002D49AD
:1004E1004E4600E47A08F608DAFC7B00740722E83D
:1004F100C0E0ECC0E0EDC0E0EEC0E0EFC0E0EA75C6
:10050100F010A4CAABF075F04DA42BFBE435F0FC60
:10051100EA2410FAEB34C5FBEC34D9FCEDC2E7FF59
:1005210075F056A4F42411C5F0F434C58FF0A42A53
:10053100E5F03BE43CF620E7141206EAD0E0FFD0F8
:10054100E0FED0E0FDD0E0FC1202AD8014F4041214
:1005510006EAD0E0FFD0E0FED0E0FDD0E0FC1205DD
:10056100B4D0E0F8E6FAEDD2E7CD33EC332482FBE8
:10057100E4C3CF33CFCE33CECD33CD33DBF37B07E3
:1005810075F00A846004F6081B0AE5F0F6088FF09E
:10059100740AA4FFACF08EF0740AA42CFEACF050E7
:1005A100010C8DF0740AA42CFDE435F0F608DBDEB5
:0305B100740722AA
:1005B400EC4D6011E8497017ED33EC3304600DE441
:1005C400FCFFFEFD22E933E8330470F802046D12E7
:1005D400043858046009E4CC2481500628500902E8
:1005E4000477284003020474C0E0EB4A7044B980E5
:1005F40006D0E0FB020463EF4E701CBD8008EBFFE5
:10060400EAFEE9FD80EBE98DF0A4FEE5F002069D2B
:10061400E9CDF9EAFEEBFFEF89F0A4FCE5F0CE8921
:10062400F0A42EFFE435F0CD89F0A42DFEE435F0DE
:100634008067EF4E7005BD80D780C3EF8BF0A4AC0C
:10064400F0EE8BF0A42CFCE435F0F8EF8AF0A42C47
:10065400E5F038FCE433CB8DF0A42CFCE5F03BF85A
:10066400EE8AF0A42CFCE5F038F8E433CF89F0A44A
:100674002CFCE5F038CF3400CE89F0A42FFFE5F050
:100684003EFEE433C98DF0A42EFEE5F039CD8AF0A8
:10069400A42FFFE5F03EFEE43DFD33D0E0FB500720
:1006A4000BBB000F020477EC2CFCEF33FFEE33FEA0
:0606B400ED33FD02044FCE
:1006BA003F8000004120000042C80000447A000048
:1006CA00461C400047C35000497424004B189680CA
:1006DA004CBEBC205A0E1BCA6753C21C749DC5AEC1
:1006EA00FB60065407601C2323120718EB5438607A
:1006FA00091207041207131205B4ECF8EDF9EEFA21
:10070A00EFCB22EB12071380F1543803241C900616
:10071A00BAFE93FC0EEE93FD0EEE930ECE93FF22DD
:030000000220D407
:0C20D400787FE4F6D8FD7581A202211B84
:10072A00BB010689828A83E0225002E722BBFE02CD
:09073A00E32289828A83E4932200
:10074300BB010CE58229F582E5833AF583E022506B
:1007530006E92582F8E622BBFE06E92582F8E222B5
:0D076300E58229F582E5833AF583E49322CF
:10077000BB010689828A83F0225002F722BBFE0168
:02078000F32262
:10078200F8BB010DE58229F582E5833AF583E8F0AD
:10079200225006E92582C8F622BBFE05E92582C859
:0207A200F22241
:1007A400BC000BBE0029EF8DF084FFADF022E4CC39
:1007B400F875F008EF2FFFEE33FEEC33FCEE9DEC02
:1007C400984005FCEE9DFE0FD5F0E9E4CEFD22ED48
:1007D400F8F5F0EE8420D21CFEADF075F008EF2F92
:1007E400FFED33FD4007985006D5F0F222C398FD83
:0507F4000FD5F0EA2220
:0E07F900C3E49FFFE49EFEE49DFDE49CFC2211
:10080700EB9FF5F0EA9E42F0E99D42F0E89C45F047
:0108170022BE
:0C081800E0FCA3E0FDA3E0FEA3E0FF2253
:10082400A8828583F0D083D08212083B12083B1241
:10083400083B12083BE473E493A3C583C5F0C58366
:10084400C8C582C8F0A3C583C5F0C583C8C582C81E
:010854002281
:10085500FAE6FB0808E6F925F0F618E6CA3AF622A4
:10086500D083D082F8E4937012740193700DA3A322
:1008750093F8740193F5828883E473740293686036
:06088500EFA3A3A380DF36
:10088B00D083D082F8E4937012740193700DA3A3FC
:10089B0093F8740193F5828883E473740293B5F033
:0D08AB00067403936860E9A3A3A3A380D89B
:102C7700EFB40A07740D122C82740A309811A899C0
:102C8700B8130CC2983098FDA899C298B811F630BD
:072C970099FDC299F5992295
:10248B008B438A448945E4F54BF54CE54A154AAE36
:10249B0049700215494E6033AB46AA47A94812074B
:1024AB002AFFAB43AA44A945054CE54CAC4B700243
:1024BB00054B14F5828C83EF120782EF60CD74010C
:1024CB002548F548E43547F54780C0AB43AA44A9F6
:0224DB00452298
:102ED900E4FFFE12072A600C0FEF70010E09E9707A
:052EE900F20A80EF2257
:1008B800E709F608DFFA8046E709F208DFFA803E22
:1008C80088828C83E709F0A3DFFA8032E309F6080F
:1008D800DFFA806EE309F208DFFA806688828C838B
:1008E800E309F0A3DFFA805A89828A83E0A3F60835
:1008F800DFFA804E89828A83E0A3F208DFFA804219
:1009080080D280FA80C680D4805580F280298010F9
:1009180080A680EA809A80A880DA80E280CA80294E
:1009280088848C8589828A83E493A30586F0A3054D
:1009380086DFF5DEF3800B89828A83E493A3F608C9
:10094800DFF9ECFAA9F0EDFB2288848C8589828A8C
:1009580083E0A30586F0A30586DFF6DEF480E3894D
:10096800828A83E493A3F208DFF980D688F0EF60E7
:10097800010E4E60CD88F0ED2402B4040050C3F59A
:1009880082EB2402B4040050B92323458223900942
:020998000873E2
:10099A00E709F60870FA8046E709F20870FA803E1D
:1009AA0088828C83E709F0A370FA8074E309F60859
:1009BA0070FA806CE309F20870FA806488828C838A
:1009CA00E309F0A370FA805889828A83E0A3F608C3
:1009DA0070FA804C89828A83E0A3F20870FA804018
:1009EA0080D280FA80C680D4805180F2802780101D
:1009FA0080A680EA809A80A880DA80E280CA80276E
:100A0A0088848C8589828A83E493A30586F0A3056A
:100A1A008670F5800B89828A83E493A3F60870F9BD
:100A2A00ECFAA9F0EDFB2288848C8589828A83E01E
:100A3A00A30586F0A3058670F680E589828A83E499
:100A4A0093A3F20870F980D888F0ED2402B4040068
:100A5A0050CEF582EB2402B4040050C4232345820D
:050A6A00239009EA736E
:1020E00002191FE493A3F8E493A34003F68001F2DE
:1020F00008DFF48029E493A3F85407240CC8C33301
:10210000C4540F4420C8834004F456800146F6DFCF
:10211000E4800B0102040810204080902F3AE47EF6
:10212000019360BCA3FF543F30E509541FFEE493C4
:10213000A360010ECF54C025E060A840B8E493A38B
:10214000FAE493A3F8E493A3C8C582C8CAC583CAB6
:10215000F0A3C8C582C8CAC583CADFE9DEE780BE6E
:012F4B000085
:00000001FF
